:10000000200D002065010000630100006301000075
:1000100000000000000000000000000000000000E0
:10002000000000000000000000000000630100006C
:1000300000000000000000006301000063010000F8
:10004000630100006301000063010000C9080000B3
:100050006301000063010000630100006301000010
:100060006301000063010000630100006301000000
:1000700063010000000000000000000063010000B8
:1000800063010000630100006301000063010000E0
:100090006301000000000000000000006301000098
:1000A00063010000630100006301000063010000C0
:1000B0000000000010B5064C2378002B07D1054B3B
:1000C000002B02D0044800E000BF0123237010BDC4
:1000D0005408002000000000B4180000084B10B5C0
:1000E000002B03D00749084800E000BF0748036819
:1000F000002B00D110BD064B002BFBD09847F9E731
:100100000000000058080020B4180000B4180000D7
:100110000000000010B5014B984710BD6D030000B2
:10012000F0B5002307E0D201C025ED05AC466244DE
:1001300054610133DBB2062B12DC012427009F40FF
:100140000722D21A865C72111F253540AC400F423F
:10015000E9D0D201C025ED05AC4662449461E8E7E0
:10016000F0BDFEE7F8B5234A234B9A4209D0224B53
:10017000204A03E011681960043304321F498B429E
:10018000F8D31F4B02E000221A6004331D4A934249
:10019000F9D31D4AFF211D4B8B439360FD399023FA
:1001A0005B001B4AD1501B4AD3780325AB43022482
:1001B0002343D370D3780C27BB4308263343D37033
:1001C000154B987B30229043202210439873997BE3
:1001D000B943314399739A7BAA4322439A730F4AD6
:1001E000516880230B4353600D4B98470D4B984744
:1001F000FEE7C046B41800000000002054080020AC
:10020000540800201C09002000ED00E00000000060
:100210000070004100500041004800410040004192
:10022000ED0D0000910C000010B5084A93692021E3
:100230000B439361064A074B5A80074B98470200CD
:1002400006490748074B984710BDC04600040040C8
:1002500004400000000C0040C508000000140040ED
:10026000D8080020E5060000F0B5C64600B5C0225B
:10027000D205102353619360254B26499962C02112
:1002800009068C4699624420195C0127B94301266E
:100290003143C9B219543221585C0F25A8430324B5
:1002A000A04644462043C0B258542020506190607C
:1002B000194898626046986245208446185CB843A5
:1002C0003043C0B264461855585C363C2040302458
:1002D000A44664462043C0B258540E3151600F4AC0
:1002E0009A620F4A9A624622995C0420814399548B
:1002F000995CB9433143C9B2995433215A5CAA433A
:1003000040460243D2B25A5404BC9046F0BDC046A7
:100310000044004110000040200000404000024026
:10032000000002C0044A136A04210B431362034A0B
:10033000034B5A807047C046000400401440000040
:10034000000C004010B5044B984704490448054B85
:100350009847054B984710BD250300000008004250
:10036000C0080020110500006902000070B5504B64
:100370009847504B40201A5C01218A431A5401309F
:100380001A5C8A431A54C022D2053D3850619060ED
:1003900049489862C0200006986242255C5D8C4303
:1003A0005C55082454619460444C9C629862013509
:1003B0005C5D8C435C55802454619460404C9C622D
:1003C000986204355C5D8C435C5580246400546104
:1003D00094603C4C9C62986201355C5D8C435C553A
:1003E0008024A40054619460374C9C62986201356B
:1003F0005C5D8C435C558024E40054619460334C14
:100400009C62986201355C5D8C435C5580242401BC
:10041000546194602E4C9C6298624B24185D884312
:1004200018550334185D884318550134185D884306
:10043000185580204002506190608020C00598626D
:10044000244C9C6206355C5D8C435C558024A40280
:10045000546194609862204C9C6201355C5D8C43D1
:100460005C558024E4025461946098621B4C9C6249
:1004700001355C5D8C435C55802424035461946099
:100480009862174C9C6201355C5D8C435C558024FE
:10049000E403546194609862124A9A6256201A5C8E
:1004A0008A431A54104B9847104B984770BDC0466A
:1004B000DD07000000440041040000400800004047
:1004C00080000040000100400002004000040040A5
:1004D00000080040010000C0020000C0040000C08D
:1004E000080000C0400000C04503000029020000D1
:1004F00010B5044B1C68044B984701002000034BC7
:10050000984710BD70080020B5070000D50700000F
:1005100070B504000D00002817D0002913D0012069
:1005200040220B490B4B98476560201D29000A4B60
:100530009847002806DB094BA382094B2361094B2E
:10054000E360002070BD0020EAE70020E8E7C04635
:10055000A817000029070000ED0800000080FFFF39
:10056000ED050000B105000030B587B004000D00B6
:10057000002815D0002911D00120B32209490A4BC7
:1005800098472B6803936B680493AB6801930593BA
:10059000201D03A9054B984707B030BD0020ECE7AC
:1005A0000020EAE7A817000029070000E90A000078
:1005B00070B584B004000E001500431E9841C0B20F
:1005C000A3220749074B984720000C3800230293C9
:1005D0000196039501A9044B984704B070BDC0462D
:1005E000A8170000290700006905000070B584B055
:1005F00004000E001500431E9841C0B2872207492F
:10060000074B984720000C3802960023019303956E
:1006100001A9044B984704B070BDC046A81700005C
:100620002907000069050000F8B50668002E02D011
:10063000330000250CE0104B984718E09F68BC463B
:100640006444A41A01348F68BC420BD21D001B689D
:10065000002B07D05C689442F0D8A41A9F68BC466F
:100660006444F0E7B34203D02800044B9847F8BD38
:10067000014B9847FBE7C04649070000750700009B
:10068000F8B50500446903695E1C0661037EDB075B
:1006900002D4037E9B070AD52B7E02221343DBB2D2
:1006A0002B76F8BD6F69E368200098473C00002C6A
:1006B000F7D06368F31AA2689342F2D32F0014377D
:1006C0003800064B9847237C012BEBD16660320043
:1006D00021003800024B9847E4E7C0467D07000040
:1006E0002906000070B504000D00002812D0002972
:1006F0000ED001203B220849084B984729002000D2
:10070000074B984700232361064B2360002070BDF0
:100710000020EFE70020EDE7C417000029070000E4
:100720006908000081060000002800D100BE704763
:100730000368002B03D08B4203D01B68F9E700202D
:1007400070470120FCE7000070B504000D00064B67
:10075000984701235840C0B239220449044B9847B6
:1007600023682B60256070BD31070000DC17000096
:100770002907000003680B60016070470368002BC5
:1007800003D01A680260180070470020FCE70000E0
:100790000300064A1268002A04D0044A1068C318ED
:1007A000136070470249014A1160F6E7740800209F
:1007B000200D002010B50300C820800058430230EF
:1007C0000321034B984783001B18580010BDC046F7
:1007D000D50C00000139FDD87047000010B5064B5C
:1007E0005A685A60054B9847054B9847054B984700
:1007F000FF20054B984710BD004000412D08000028
:10080000FD0B0000410C00000D080000C3070AD5D5
:10081000054B802252009A60832252025A60024B9A
:100820005B78DB09FBD17047000C0040064B1A7A5D
:10083000D2B21A725A7AD2B25A729A7AD2B29A72E0
:10084000DA7AD2B2DA7270470004004010B50400C0
:10085000C3681B7ADB0706D50368002B00D09847D6
:10086000E36801221A7210BD70B504000D00431E2A
:100870009841C0B233221049104B9847E5600123DC
:100880002B80AB7ADB09FCD1E268937ADB09FCD1DF
:1008900080331380937ADB09FCD1E268936980236B
:1008A000DB009361937ADB09FCD10133E268D371F9
:1008B000034B1C60002070BDFC17000029070000DE
:1008C000780800200020704710B5024B1868024BD2
:1008D000984710BD780800204D080000024B9C4648
:1008E0006044800AC0B2704700F8FFBD70B50600D2
:1008F0000C000800714B98470023002B00D184E0C6
:100900000025002E00D18DE0002C00D188E00120D0
:100910006B4A6C496C4B9847002D00D1CBE0E369E2
:10092000DB0721D42A786B781B021343AA781204C0
:100930001343EA7812061A431C231A40E3699B0703
:10094000FCD123689B0709D5236802218B432360D0
:10095000E3699B07FCD1E3699B07FCD401231343A4
:100960002360E3699B07FCD1E369DB07FCD43460B7
:100970002B786A7812021A43AB781B041A43EB787F
:100980001B0613431C221340082B4DD0002C00D112
:100990008DE0002D00D188E001204C4A49494A4BA6
:1009A00098472B786A7812021A43AB781B041A43D3
:1009B000EB781B061343464A13402360E3699B0709
:1009C000FCD12B796A7912021A43AB791B041A43C2
:1009D000EB791B0613433F4A1340802292021343D4
:1009E0006360E3695B07FCD12B7B23736A7B302355
:1009F000E2542B795B075CD101233371AA7BEB7B3B
:100A00001B021343F380002070BD002802D0013385
:100A1000DBB272E71D01EA182F4D3C35AD1870E7C7
:100A2000002075E7002073E7002C3CD0002D38D063
:100A300001202A4A2349244B98472B786A781202CE
:100A40001A43AB781B041A43EB781B061343204A66
:100A500013402360E3699B07FCD12B796A7912026A
:100A60001A43AB791B041A43EB791B0613431C4A48
:100A700013401C4A13436360E3695B07FCD12B7A84
:100A80006A7A12021A43AB7A1B041A43EB7A1B06EA
:100A9000134363626A7B3023E254E369002BFCD189
:100AA000A7E70020C5E70020C3E7002075E7002086
:100AB00073E70223A1E70D204042A5E7DD0800000F
:100AC000250900006418000029070000EF08000055
:100AD000FCFEFFFFBF1DFDFF14180000030900000E
:100AE000BFDDFDFF40020200F0B5CE46474680B5AF
:100AF00089B081460D0004680B6803934B6804932A
:100B00000023059306930679002814D0002C10D0FA
:100B10000120374A3749384B9847E3695B0764D16E
:100B2000E3699B07FCD123689B0720D41420404233
:100B300056E00020EDE70020EBE700222DE04878AA
:100B4000000247460743B84602310391013205923D
:100B50004246A2625BB2002B35DB002000283ADB64
:100B60000598AB68984202D3069A934233D9237E04
:100B7000DBB25A07E1D5A16A049A002A08D0501CBA
:100B800004901170012E03D9901C0490090A517031
:100B9000069A0192013206920122002ADAD10699C0
:100BA000059A9142D6D34946C888D907D2D5039928
:100BB000002906D0481C039008788046012EBED834
:100BC000C4E78046C2E701235B4263838133237617
:100BD00013204042C2E7237E9B07FCD003232376E9
:100BE00009B00CBC90469946F0BD04204042F7E79E
:100BF000850A000064180000290700000E4A116AE7
:100C0000090C136A9B0F9B0709040C4801400B4316
:100C100002210B43136293690B439361137F1D31D0
:100C20000B401377044BDB681B07FBD5024A136AA2
:100C300080210B4313627047000800400000FF0F43
:100C4000024A936902218B43936170470008004078
:100C5000F8B50C4D202128000B4CA047FA277F0047
:100C600038000A4EB04724212800A0473800B0477A
:100C700001212800A0473800B04700212800A047E4
:100C8000F8BDC0460000002021010000F104000072
:100C900010B5034B9847034B9847024B9847FCE726
:100CA00015010000510C000070B59E25084C2D0167
:100CB0002800E56000F0C2F8A060002804D00023FE
:100CC00060600560436070BDE0606060FBE7C04647
:100CD0007C080020002243088B4274D303098B4216
:100CE0005FD3030A8B4244D3030B8B4228D3030CFC
:100CF0008B420DD3FF22090212BA030C8B4202D39E
:100D00001212090265D0030B8B4219D300E0090AC5
:100D1000C30B8B4201D3CB03C01A5241830B8B42CE
:100D200001D38B03C01A5241430B8B4201D34B03B7
:100D3000C01A5241030B8B4201D30B03C01A52411C
:100D4000C30A8B4201D3CB02C01A5241830A8B42A1
:100D500001D38B02C01A5241430A8B4201D34B028A
:100D6000C01A5241030A8B4201D30B02C01A5241EE
:100D7000CDD2C3098B4201D3CB01C01A52418309A2
:100D80008B4201D38B01C01A524143098B4201D3DC
:100D90004B01C01A524103098B4201D30B01C01A07
:100DA0005241C3088B4201D3CB00C01A5241830881
:100DB0008B4201D38B00C01A524143088B4201D3AE
:100DC0004B00C01A5241411A00D20146524110460E
:100DD0007047FFE701B5002000F006F802BDC046ED
:100DE0000029F7D076E770477047C04670B50D4EC2
:100DF0000D4D0024AD1BAD1005D0A300F3580134F8
:100E00009847A542F9D100F03DFD084E084D002459
:100E1000AD1BAD1005D0A300F35801349847A5428F
:100E2000F9D170BD901800009018000090180000D3
:100E30009C1800007047C0467047C04610B5034B71
:100E40000100186800F004F810BDC0461000002032
:100E5000F0B557464546DE464E46E0B50D000B352B
:100E600083B00700162D00D89FE007239D4300D5CF
:100E7000C4E0A94200D9C1E000F09EFAF823FF3394
:100E80009D4200D88FE2680A00D1BBE0042800D957
:100E900062E138239846A80980443930C100D24E17
:100EA00071180839CC68A14219D0032362689A43AB
:100EB0001300521B0F2A00DDAAE0002A00DB88E0A5
:100EC00003239C4608E06246636893435A1B0F2A3B
:100ED00000DD9DE0002A7CDAE468A142F3D1320013
:100EE00034690832944200D190E103236168994348
:100EF0008946491B0F2900DD62E1726132610029D8
:100F000000DB87E0B94A4B46914500D930E1DB0868
:100F1000FF3A9910FF3A8A40DB0071689B190A4337
:100F200099687260E360A1609C601300CC6001214D
:100F30008210914099426FD80B4205D10322904311
:100F4000490004300B42FBD003239846C300994666
:100F5000B144CC4682466346DC68A44507D157E1DC
:100F6000002A00DB66E1E468A44500D150E1424676
:100F7000636893435A1B0F2AF2DD012080466119F2
:100F800005436560A068E5680836C560A86040460E
:100F9000F160B16010434860CE608E603800E2506E
:100FA00000F012FA2000083021E0102926D838007D
:100FB00000F002FA1025182302208B4EF3181A00B5
:100FC0005C68083A944200D12EE1032362689A4398
:100FD0001300E268A168CA6091600122E3185968B1
:100FE00038000A435A6000F0EFF92000083003B0DF
:100FF0003CBC90469946A246AB46F0BD0C2300206F
:101000003B60F4E780213F2340208900984646E773
:10101000404664E74B46E0E70323B46862689A43BE
:101020009046AA4203D3531B0F2B00DD86E023001A
:1010300043446F4A01936F4B93461B681268EB1849
:10104000013200D168E16C4A944663441B0B1B03D8
:1010500000930099380000F0BFF903008146013386
:1010600061D0019B834200D9FFE0644B009A9A460D
:101070001B689C46534662441A60019B11008342E0
:1010800000D155E15B461B68013300D16CE14B4652
:10109000019A9B1A59185346196007234A46134070
:1010A00000D124E1082189465549D21A9144CB1A2E
:1010B000009A38004A441105090D5B1A19009B4635
:1010C00000F08AF9431C00D142E14B46C01A0123CB
:1010D0005844184353461B685B4419005346196033
:1010E0004B46B3605860B44213D043460F2B00D830
:1010F000E8E04346072260680C3B9343063A02400F
:1011000005201A436260E218506090600F2B00D9EE
:1011100022E13C4B1A68914200D919603A4B1A6897
:10112000914200D919600323B46862689A43531B43
:10113000954200D9C9E00F2B00DCC6E0012229004E
:1011400013431143651961603800B5606B6000F0AE
:101150003BF9200008304AE714287AD9542800D9EE
:10116000BAE06E239846280B80446F30C10096E6A3
:101170005A0A042A73D9142A00D9D0E011005C322B
:101180005B31D20008235B429C46B218944463460C
:101190009A6803239846944500D1ABE043465168D2
:1011A0009943894500D395E092689445F6D163460A
:1011B000DA6873686146E260A1609460CC60B6E66C
:1011C000012360191D43656070613061C2608260F7
:1011D0001A004B460A4342603800E15000F0F4F830
:1011E0002000083003E7C04640040020FF01000053
:1011F00048080020BC0800200F1000008C080020C8
:1012000008100000B4080020B808002073688EE6BB
:1012100008239B46073BDC449B46DA444346524640
:10122000134200D097E637E0DC680230A34200D1D9
:1012300055E6CAE60122E318596838000A435A60A5
:10124000E368A268D3609A6000F0BEF8200008301E
:10125000CDE65B23984680445C30C1001FE69A09C6
:10126000110039323831D2008CE7B44200D05AE74D
:101270004F4B009A9A461B689C46534662441100A5
:101280001A60FFE608235B429C46E1444B469B689C
:101290000138994500D084E043460342F2D1736897
:1012A0008B4373604900994200D9B5E6002900D10B
:1012B000B2E650460B4200D048E6490004300B42EB
:1012C000FBD043E601234A465360380000F07CF827
:1012D00000208CE694466AE7AA235B00984211D866
:1012E000DD3B9846E80B80447830C100D7E5802389
:1012F0005B01DDE68910023B8B407268134373602B
:10130000624657E72B4B98421CD87C239846A80C82
:1013100080447D30C100C2E51033009399E6542A21
:1013200026D84B461A0B11006F326E31D20029E7D6
:101330001B0500D0A6E60120009BB268434403438E
:101340005360E6E6FE217E237F2089009846A6E5CD
:10135000002301209B46BDE621003800083100F043
:10136000CBF853461968D4E65B464A461A6094E6C1
:10137000AA2149008A4206D84B46DA0B110078327E
:101380007731D200FEE60B498A4206D84B469A0CCA
:1013900011007D327C31D200F4E6FE227E219200E3
:1013A000F0E673687EE72B00E808083305E6C046E0
:1013B0008C0800205405000010B50248FFF73AFDE4
:1013C00010BDC0460409002010B50248FFF734FDE7
:1013D00010BDC04604090020002370B5064C05006E
:1013E00008002360FFF7D4F9431C00D070BD2368C8
:1013F000002BFBD02B60F9E718090020034B10B538
:10140000002B02D0024800F005F810BD00000000DB
:101410002514000010B5010000230022002000F078
:1014200049F910BD70B5094B094CE41AA41009D054
:10143000084AA518AD00ED182B68013C9847043DFB
:10144000002CF9D100F02AFA70BDC046A81800009F
:10145000AC180000FFFFFF3FF8B50C000600FFF7D7
:10146000ABFF204FBB685D6803239D431E4B2C1BC5
:101470009C466444240B1D4B013C24039C4207DD25
:1014800000213000FFF7A8FFBB685B19984204D029
:101490003000FFF799FF0020F8BD61423000FFF7F0
:1014A0009BFF431C0DD00122BB682D1B15435D60C3
:1014B0000F4B30001A68141B1C60FFF785FF0120DA
:1014C000EAE700213000FFF787FFBA68831A0F2B85
:1014D000DEDD08490968401A0549086001210B430F
:1014E0005360D5E740040020EF0F0000FF0F00001D
:1014F0008C08002048080020F8B504000D1E3CD0E0
:10150000FFF75AFF29000839486801230500032620
:101510009D434A199C46614F5368B343BE68B2422B
:1015200056D06646536006420AD13E000868083627
:10153000091A2D188868B04265D0CE68C660B060C0
:101540000120D6187668064233D0554B28434860B0
:101550004D519D4212D8ED08FF3BAA10FF3B93402E
:101560007A68ED0013437B60EF19BB68CF608B6036
:10157000B960D9602000FFF727FFF8BD680A04288A
:1015800050D8A809020039303832C000381808385D
:101590008368032698424CD05A68B243954230D2B1
:1015A0009B689842F8D1C368CB6088609960C1603D
:1015B000E0E7ED183B4E9368B34242D0D26828432F
:1015C000DA609360364B48604D519D42D6D8C2E7F1
:1015D0006246EB18024206D10A68891A88689B188D
:1015E000CA68C260906001221A434A602E4AB960FC
:1015F00012689342BED32D4B20001968FFF72CFFD1
:10160000B8E71800CFE76646D018406830423FD1AF
:1016100090685D19D368C360986063462B434B6044
:101620004D51A7E7142814D802005C305B32C0008B
:10163000ACE70123921093407A6813437B60030068
:10164000B2E72843D9609960CB608B6048604D5108
:1016500090E7542805D8280B02006F306E32C00086
:1016600094E7AA225200904205D8E80B0200783095
:101670007732C0008AE70E4A904205D8A80C0200D3
:101680007D307C32C00081E7FE207E2280007DE735
:1016900063462B434B6015606CE7C0464004002056
:1016A000FF010000480400204C080020BC08002076
:1016B00054050000F0B54E464546DE465746E0B5B7
:1016C000364D83B00600286898460F009146FFF714
:1016D000B1FB334B1C68A4235B00E058002852D0B8
:1016E00043681F2B13DC5A1C0192002E28D1019A4B
:1016F00002339B0042601F502868FFF79DFB0020CB
:1017000003B03CBC90469946A246AB46F0BD254B83
:10171000002B3DD0C8204000FFF790FB002837D0B9
:10172000A42200235200A15843600160A05040321F
:10173000835004328350013301930023002ED6D00E
:101740009A00924682444A46882154466250C422F6
:101750005200914681444A468739994012688B4627
:101760000A4394464A46614611608422414652002B
:10177000A150022EBBD102005C468D32FF321168AF
:101780000C431460B3E720004D30FF30E050A7E772
:101790002868FFF751FB01204042B1E750080020C4
:1017A000801800003D0E00002E2E2F68616C2F73F4
:1017B00072632F68616C5F7370695F6D5F73796EC0
:1017C000632E63002E2E2F68616C2F7372632F6857
:1017D000616C5F74696D65722E6300002E2E2F6838
:1017E000616C2F7574696C732F7372632F757469D4
:1017F0006C735F6C6973742E630000002E2E2F686B
:10180000706C2F7274632F68706C5F7274632E63D8
:1018100000000000000000000000000000000000C8
:1018200000000000000000000000000000000000B8
:1018300000000000000000000000000000000000A8
:101840000000000000000000000000000000000098
:101850000C00200000000200000000004F00FF010B
:10186000000000002E2E2F68706C2F736572636F5E
:101870006D2F68706C5F736572636F6D2E6300000F
:1018800018000020F8B5C046F8BC08BC9E4670475A
:10189000FD130000DD000000A90C0000F8B5C046F3
:0C18A000F8BC08BC9E467047B500000074
:0818AC00FCF3FF7F01000000C6
:1018B4001211100908070B0A1211100908070B0A64
:1018C40018000020000000000000000004030020B5
:1018D4006C030020D403002000000000000000007E
:1018E40000000000000000000000000000000000F4
:1018F40000000000000000000000000000000000E4
:1019040000000000000000000000000000000000D3
:1019140000000000000000000000000000000000C3
:1019240000000000000000000000000000000000B3
:1019340000000000000000000000000000000000A3
:101944000000000000000000000000000000000093
:101954000000000000000000000000000000000083
:101964000000000000000000000000000000000073
:1019740001000000000000000E33CDAB34126DE610
:10198400ECDE05000B000000000000000000000079
:101994000000000000000000000000000000000043
:1019A4000000000000000000000000000000000033
:1019B4000000000000000000000000000000000023
:1019C4000000000000000000000000000000000013
:101CF4000000000000000000400400204004002018
:101D0400480400204804002050040020500400200F
:101D140058040020580400206004002060040020BF
:101D2400680400206804002070040020700400206F
:101D3400780400207804002080040020800400201F
:101D440088040020880400209004002090040020CF
:101D54009804002098040020A0040020A00400207F
:101D6400A8040020A8040020B0040020B00400202F
:101D7400B8040020B8040020C0040020C0040020DF
:101D8400C8040020C8040020D0040020D00400208F
:101D9400D8040020D8040020E0040020E00400203F
:101DA400E8040020E8040020F0040020F0040020EF
:101DB400F8040020F804002000050020000500209D
:101DC400080500200805002010050020100500204B
:101DD40018050020180500202005002020050020FB
:101DE40028050020280500203005002030050020AB
:101DF400380500203805002040050020400500205B
:101E0400480500204805002050050020500500200A
:101E140058050020580500206005002060050020BA
:101E2400680500206805002070050020700500206A
:101E3400780500207805002080050020800500201A
:101E440088050020880500209005002090050020CA
:101E54009805002098050020A0050020A00500207A
:101E6400A8050020A8050020B0050020B00500202A
:101E7400B8050020B8050020C0050020C0050020DA
:101E8400C8050020C8050020D0050020D00500208A
:101E9400D8050020D8050020E0050020E00500203A
:101EA400E8050020E8050020F0050020F0050020EA
:101EB400F8050020F8050020000600200006002098
:101EC4000806002008060020100600201006002046
:101ED40018060020180600202006002020060020F6
:101EE40028060020280600203006002030060020A6
:101EF4003806002038060020400600204006002056
:101F04004806002048060020500600205006002005
:101F140058060020580600206006002060060020B5
:101F24006806002068060020700600207006002065
:101F34007806002078060020800600208006002015
:101F440088060020880600209006002090060020C5
:101F54009806002098060020A0060020A006002075
:101F6400A8060020A8060020B0060020B006002025
:101F7400B8060020B8060020C0060020C0060020D5
:101F8400C8060020C8060020D0060020D006002085
:101F9400D8060020D8060020E0060020E006002035
:101FA400E8060020E8060020F0060020F0060020E5
:101FB400F8060020F8060020000700200007002093
:101FC4000807002008070020100700201007002041
:101FD40018070020180700202007002020070020F1
:101FE40028070020280700203007002030070020A1
:101FF4003807002038070020400700204007002051
:102004004807002048070020500700205007002000
:1020140058070020580700206007002060070020B0
:102024006807002068070020700700207007002060
:102034007807002078070020800700208007002010
:1020440088070020880700209007002090070020C0
:102054009807002098070020A0070020A007002070
:10206400A8070020A8070020B0070020B007002020
:10207400B8070020B8070020C0070020C0070020D0
:10208400C8070020C8070020D0070020D007002080
:10209400D8070020D8070020E0070020E007002030
:1020A400E8070020E8070020F0070020F0070020E0
:1020B400F8070020F807002000080020000800208E
:1020C400080800200808002010080020100800203C
:1020D40018080020180800202008002020080020EC
:1020E400280800202808002030080020300800209C
:1020F4003808002038080020FFFFFFFF000002001E
:04210400F4080020BB
:00000001FF
